:020000021000EC
:10F800000C9446FC0C9463FC0C9463FC0C9463FC19
:10F810000C9463FC0C9463FC0C9463FC0C9463FCEC
:10F820000C9463FC0C9463FC0C9463FC0C9463FCDC
:10F830000C9463FC0C9463FC0C9463FC0C9463FCCC
:10F840000C9463FC0C9463FC0C9463FC0C9463FCBC
:10F850000C9463FC0C9463FC0C9463FC0C9463FCAC
:10F860000C9463FC0C9463FC0C9463FC0C9463FC9C
:10F870000C9463FC0C9463FC0C9463FC0C9463FC8C
:10F880000C9463FC0C9463FC0C9463FC11241FBE69
:10F89000CFEFD0E1DEBFCDBF11E0A0E0B1E0E2E804
:10F8A000FFEF01E00BBF02C007900D92A430B1073B
:10F8B000D9F712E0A4E0B1E001C01D92A634B1076F
:10F8C000E1F70C9483FF0C9400FC0F92AF93BF936D
:10F8D000CF93DF93EF93FF93FC01EA01DB01D8950F
:10F8E000099231961197D9F7FF91EF91DF91CF915E
:10F8F000BF91AF910F9008950F921F920F93AF9306
:10F90000BF93CF93DF93EF93FF93FC01EA01DB01F9
:10F910000990199001E043D032961297C9F7FC0183
:10F9200003E03DD005E03BD0FF91EF91DF91CF9117
:10F93000BF91AF910F911F900F9008950F931F9358
:10F94000EF93FF93FC0103E02AD000E011E0E00F09
:10F95000F11FE617F707B9F7FF91EF911F910F918C
:10F9600008950F930F9222D0082E09E018D00F901F
:10F970000F9108950F930F92EF93FF9317D0FC010F
:10F9800060936800C895802DFF91EF910F900F91C3
:10F9900008950F930BD001E102D00F910895E199E2
:10F9A000FECF00936800E895FFFF0000009168001B
:10F9B00000FDFCCF089587E089B98AB188618AB9D2
:10F9C00008958AB1877E8AB908958CB95E9BFECF6F
:10F9D0005E9A08958CB1992708958BB19927807804
:10F9E00090700895EF92FF920F931F93CF93DF9340
:10F9F0007B01C0E0D0E0C617D70770F48C010E94ED
:10FA0000EDFC8823E1F30E94EAFCF80181938F0169
:10FA10002196CE15DF0598F381E090E0DF91CF913C
:10FA20001F910F91FF90EF900895EF92FF920F9327
:10FA30001F93CF93DF937C018B01C0E0D0E0C01710
:10FA4000D10738F4F70181917F010E94E5FC2196EE
:10FA5000F6CF81E090E0DF91CF911F910F91FF9061
:10FA6000EF900895EF92FF920F931F93CF93DF9340
:10FA70007C0100E010E00817190788F4C0E0D0E02E
:10FA800000000E94EDFC882351F4219687E0C335E5
:10FA9000D807B0F30F5F1F4F0E151F0578F3DF91E6
:10FAA000CF911F910F91FF90EF9008950E94E1FC7C
:10FAB0000E9400000895DF92EF92FF920F931F9330
:10FAC000CF93DF93CDB7DEB72197DEBFCDBF8C01DB
:10FAD0007B011982D98061E070E0CE01860F971F0B
:10FAE0000E94F2FC89818B31B1F761E070E0C801BE
:10FAF0000E94F2FC61E070E0CE01860F971F0E9429
:10FB0000F2FC89819927182F002761E070E0CE016F
:10FB1000860F971F0E94F2FC8981080F111D61E07A
:10FB200070E0CE01860F971F0E94F2FC89818E3013
:10FB3000B9F4C8010196BC01C7010E94F2FC98010A
:10FB40008FEF0F3F180779F0F70181917F01D826D9
:10FB500021503040FFEF2F3F3F07B1F7DD2019F074
:10FB600080E090E001C0C8012196DEBFCDBFDF91EB
:10FB7000CF911F910F91FF90EF90DF900895CF925A
:10FB8000DF92FF920F931F93CF93DF93182FEB0118
:10FB90006A018BE10E94E5FC4BE1F42E812F0E946B
:10FBA000E5FCF1260D2F1127802F0E94E5FCF026A1
:10FBB0008C2F0E94E5FCFC268EE00E94E5FC8EE086
:10FBC000F82621978FEFCF3FD80759F0F6018191A2
:10FBD0006F01F8260E94E5FC2197FFEFCF3FDF077A
:10FBE000A9F78F2D0E94E5FCDF91CF911F910F9116
:10FBF000FF90DF90CF90089599278139910559F0B2
:10FC00008239910524F48039910529F008C08239A0
:10FC1000910519F004C082E003C087E001C080ECC8
:10FC200099270895BF92CF92DF92EF92FF920F93A0
:10FC30001F93CF93DF93B82E8B01FB018081C82FD8
:10FC4000DD27C231D10509F46DC0C331D105DCF423
:10FC5000C330D10509F44DC0C430D10544F4C130DE
:10FC6000D10579F1C230D10509F44AC018C1C630B6
:10FC7000D10509F44AC0C630D1050CF410C1609713
:10FC80000CF40DC154C0C531D10509F4DCC0C63136
:10FC9000D10544F4C331D10509F47CC0649709F45B
:10FCA00049C0FDC0CA31D10509F4EBC0CB31D10543
:10FCB00024F4669709F4AEC0F2C06B9709F4D8C07B
:10FCC000EEC0FB01118288E0828381E4838386E5B4
:10FCD000848382E5858389E4868383E5878380E561
:10FCE00080878FE5818782E38287AB016BE070E0DC
:10FCF000DCC0FB0181810E94FCFDF801828301C010
:10FD0000FB011182A801BE01D0C0FB0183819927AC
:10FD1000982F88272481820F911D9093450280930C
:10FD2000440206C060E070E0CB010E949EFCF80136
:10FD30001182B8C0FB0181819927D82FCC278281FD
:10FD40009927C82BD92B809144029091450297FFA7
:10FD500003C081E08BBF01C01BBEF8011182C80146
:10FD600002962091440230914502AC01BE01C901C6
:10FD7000880F991F0E9465FCF801EC0FFD1F12828D
:10FD80009E01369527958091440290914502820FFD
:10FD9000931F53C0FB0181819927D82FCC278281E3
:10FDA0009927C82BD92B809144029091450297FF47
:10FDB00003C081E08BBF01C01BBECC24DD24CC1668
:10FDC000DD06D8F4FAE0EF2EF12CE00EF11E809162
:10FDD000440290914502880F991FA70160E071E0ED
:10FDE0008C0D9D1D0E947CFC80E091E0C80ED91E08
:10FDF000E80EF91ECC16DD0650F30E94C9FCF8018E
:10FE00001182D695C79580914402909145028C0F3E
:10FE10009D1F29C0FB0181819927D82FCC27828182
:10FE20009927C82BD92B1182EC0FFD1F12828091CC
:10FE30004402909145028C0F9D1F90934502809340
:10FE4000440223965FCFFB0181819927382F222717
:10FE500082819927282B392B11828091440290911D
:10FE60004502820F931F90934502809344021AC06B
:10FE7000FB0111828481E82FFF27E050FF4F808132
:10FE800007C0FB01118269E081E090E00E94BAFCAA
:10FE9000F80182831382A80164E070E006C089EC57
:10FEA000F8018183A80162E070E08B2D0E94BFFD04
:10FEB000DF91CF911F910F91FF90EF90DF90CF9046
:10FEC000BF900895CF93DF93CDB7DEB72197DEBF04
:10FED000CDBF69E081E090E00E94BAFC992784FFE1
:10FEE00009C08F7E0E94B1FC05C064E071E0898189
:10FEF0000E9412FE64E071E0CE0101960E945BFD5B
:10FF0000892B99F3F7CFCFEFD0E1DEBFCDBFCEE1A4
:10FF1000F894AEEFBFE00E94B8FF802D843B79F4E7
:10FF2000AFEFBFE00E94B8FF802D833C41F4ADEFFE
:10FF3000BFE00E94B8FF802D992780936F000E9438
:10FF4000DBFC0E94EAFC84E690E00E9432FD0E9405
:10FF5000EDFC882319F00E9462FF04C0C150C8BBA9
:10FF6000CC2389F70E9456FD80E090E00C94C0FFFE
:10FF7000E199FECFBFBBAEBBE09A11960DB20895DA
:02FF8000FFCFB1
:04FF82001E970200C4
:040000031000F800F1
:00000001FF
